:020000020000FC
:100000000FED0DBF0FEF01BB0BD030D038D040D07B
:1000100048D050D058D060D068D070D078D0FFCFC2
:1000200000E083D00DE381D09098919A81D091988F
:100030007FD00DE37AD0919A7BD0919879D002E06D
:1000400074D0919875D0089503E06FD0919870D0D6
:1000500003E06BD091986CD0089507E266D0919838
:1000600067D007E162D0919863D008950FE15DD029
:1000700091985ED00FE159D091985AD0089503E03D
:1000800054D0919855D00BE150D0919851D008950B
:100090000FE34BD091984CD003E147D0919848D0D2
:1000A00008950FE242D0919843D00BE13ED0919851
:1000B0003FD0089503E239D091983AD00FE135D07E
:1000C000919836D008950FE230D0919831D00FE05A
:1000D0002CD091982DD008950FE327D0919828D057
:1000E0000FE023D0919824D0089507E01ED0919876
:1000F0001FD00BE11AD091981BD008950FE315D0B3
:10010000919816D00FE111D0919812D008950FE276
:100110000CD091980DD00FE108D0919809D0089596
:1001200002E003D0919804D0089502BB01D0089555
:0801300018EC1A95F1F708958F
:00000001FF
